:020000040000FA
:0600000041EF21F01200A7
:020006001200E6
:060008005DEF08F012009C
:06001800ECEF00F0120005
:02001E000100DF
:0C0020009E42000000010000B70000003C
:04002C00948E949C7E
:10003000200EAF6EAC8AAC84AC9CAB8EAB889E9825
:100040009D8AF28EF28C1200D9CFE6FFE1CFD9FF64
:10005000E65200016251601902E16351611901E148
:10006000F8D760C0E9FF61C0EAFF602B000E612392
:10007000EFCFDFFF280E605D010E615904E3000E33
:10008000606F010E616FDF5000D0E552E552E7CF9F
:10009000D9FF1200D9CFE6FFE1CFD9FF020EE1264A
:1000A000DE6ADD6AACB210D0DF2A010E01E3DB2A82
:1000B000D9CFE9FFDACFEAFFE80ED880EE54030E7D
:1000C000ED5401E206D0EED7FE0EDB50AD6E9EA8D9
:1000D000FED7020EE15C02E2E16AE552E16EE55212
:1000E000E7CFD9FF1200D9CFE6FFE1CFD9FF030E4A
:1000F000E126FD0EDBCFDEFFDBCFDDFFA5DFE76E08
:10010000020EE7CFDBFFFC0EDB50F36E020EDB507E
:10011000F35C0DE0FD0EDBCFE9FFDB2AFE0EDBCF4B
:10012000EAFF01E3DB2A020EDBCFEFFFE7D7FD0E8C
:10013000DBCFE9FFFE0EDBCFEAFFEF6ADECF00F098
:10014000DDCF01F000C0F3FF01C0F4FF030EE15C5E
:1001500003E200D0E16AE552E16EE552E7CFD9FF54
:100160001200D9CFE6FFE1CFD9FF020EE126DE6A09
:10017000DD6AFD0EDBCFE9FFFE0EDBCFEAFFEF50BD
:1001800014E0FD0EDBCFE9FFFE0EDBCFEAFFEF5000
:10019000E66E80DFE552DF2A010E01E3DB2AFD0E69
:1001A000DB2AFE0E01E3DB2AE4D7010EF36EF46ACC
:1001B000020EE15C03E200D0E16AE552E16EE55235
:1001C000E7CFD9FF12000D0EE66E64DFE5520A0E8E
:1001D000E66E60DFE5521200DACFE4FFE2CFDAFF2D
:1001E000E9CFE4FFEACFE4FFE652D9CFE6FFE1CF63
:1001F000D9FFE6529EAA16D0AE50DF6E000162C053
:10020000E9FF63C0EAFF622B000E6323DFCFEFFF3D
:10021000280E625D010E635904E3000E626F010E49
:10022000636F9E9AE552E552E7CFD9FFE552E5CFDD
:10023000EAFFE5CFE9FFE5CFDAFF1100D9CFE6FF0E
:10024000E1CFD9FFFE0EDB50000803E2FE0EDB0615
:10025000F9D7E552E7CFD9FF1200D9CFE6FFE1CFBA
:10026000D9FFFE0EDBCFE6FF08EC21F0E552E552A8
:10027000E7CFD9FF1200D9CFE6FFE1CFD9FF030EB8
:10028000E126FE0EDB505F0801E26ED0FD0EDB5072
:100290003F0801E269D0FE0EDBCFE6FFFD0EDB502A
:1002A000F80BE842E842E842600DF350E552E724DB
:1002B000DE6EDD6AFD0EDBCFE6FFDB50F80BE842B9
:1002C000E842E842080DF350E552E75CE76E020EA3
:1002D000E7CFDBFFFC0EDB5016E1010EF36E020EE2
:1002E000DB5004E0D890F336E806FCE1F350E81C5C
:1002F000006EDECFE9FFDDCFEAFF830EE926000EB8
:10030000EA220050EF16FC0EDB0415E1010EF36E3D
:10031000020EDB5004E0D890F336E806FCE1F3501F
:10032000006EDECFE9FFDDCFEAFF830EE926000E87
:10033000EA220050EF12FC0EDB50020815E1010E1C
:10034000F36E020EDB5004E0D890F336E806FCE1D1
:10035000F350006EDECFE9FFDDCFEAFF830EE92622
:10036000000EEA220050EF1A030EE15C02E2E16A9D
:10037000E552E16EE552E7CFD9FF1200D9CFE6FF93
:10038000E1CFD9FF0A0EE126FB0EDBCFE6FFFD0E23
:10039000DB50E552E75CE66ED950020FE96EDACF2A
:1003A000EAFFE552E750EE6EED6AFC0EDBCFE6FFAA
:1003B000FE0EDB50E552E75CDE6EDD6A020EDBCF3F
:1003C00000F0030EDBCF01F00001800E011415E0F8
:1003D00020682168020EDBCF25F0030EDBCF26F06C
:1003E0001AEC16F0020E1EC0DBFF030E1FC0DBFF6F
:1003F000060EDB68070EDB6807D0010EF36E060EF3
:10040000F3CFDBFF070EDB6ADECF00F0DDCF01F0BC
:100410000001800E011411E020682168DECF25F074
:10042000DDCF26F01AEC16F01EC0DEFF1FC0DDFF88
:10043000040EDB68050EDB6807D0010EF36E040EB8
:10044000F3CFDBFF050EDB6AD9CFE9FFDACFEAFF96
:10045000010ED890EE36ED36E806FBE1D950020FDA
:10046000E96EDACFEAFF010ED890EE36ED36E806F7
:10047000FBE1FA0EDBCFE6FFFD0EDBCFE6FFFE0E63
:10048000DBCFE6FFF8DEE552E552E552DECF00F0C5
:10049000DDCF01F0020EDBCF02F0030EDBCF03F065
:1004A00003500118E8AE02D0013404D00050025CC1
:1004B0000150035867E2DECF02F0DDCF03F0D890A1
:1004C00003320232020EDBCF20F0030EDBCF21F02D
:1004D0000250205C006E03502158016E080E00C0CF
:1004E000DBFF090E01C0DBFFFC0EDB50F36EFE0EDE
:1004F000DB50F35C46E0080EDBCF00F0090EDBCFEB
:1005000001F00001800E011416E1FD0EDBCFE7FFC4
:10051000060EDB50E726FD0EE7CFDBFFDECF00F057
:10052000DDCF01F0D950080FE96EDACFEAFF0050B5
:10053000EE5E0150ED5AFE0EDBCFE7FF040EDB50FE
:10054000E726FE0EE7CFDBFF020EDBCF00F0030E47
:10055000DBCF01F0D950080FE96EDACFEAFF005087
:10056000EE260150ED22FA0EDBCFE6FFFD0EDBCFCB
:10057000E6FFFE0EDBCFE6FF7EDEE552E552E552FA
:10058000B3D762D0020EDBCF02F0030EDBCF03F055
:10059000D890033202320250DE5C006E0350DD5808
:1005A000016E080E00C0DBFF090E01C0DBFFFB0E71
:1005B000DB50F36EFD0EDB50F35C46E0080EDBCF44
:1005C00000F0090EDBCF01F00001800E011418E1EC
:1005D000FE0EDBCFE7FF040EDB50E726FE0EE7CF73
:1005E000DBFF020EDBCF00F0030EDBCF01F0D950B2
:1005F000080FE96EDACFEAFF0050EE5E0150ED5AC7
:10060000FD0EDBCFE7FF060EDB50E726FD0EE7CF42
:10061000DBFFDECF00F0DDCF01F0D950080FE96E2F
:10062000DACFEAFF0050EE260150ED22FA0EDBCFC2
:10063000E6FFFD0EDBCFE6FFFE0EDBCFE6FF1BDEA7
:10064000E552E552E552B3D70A0EE15C02E2E16AF7
:10065000E552E16EE552E7CFD9FF1200D9CFE6FFB0
:10066000E1CFD9FF020EE126E66AE66A50DAE552EA
:10067000E55201012B6B2C6BDE6ADD6ADECF00F0E8
:10068000DDCF01F0000E005C030E015811E2DECF59
:10069000E9FFDDCFEAFF830EE926000EEA22EF50E4
:1006A000E66EF3D9E552DF2A010E01E3DB2AE6D735
:1006B000020EE15C02E2E16AE552E16EE552E7CF4B
:1006C000D9FF1200D9CFE6FFE1CFD9FFFA0EDBCF79
:1006D000E6FFFD0EDBCFE6FFFC0EDBCFE6FFFD0EF7
:1006E000DBCFE6FFFE0EDBCFE6FF48DE006E050E39
:1006F000E15E0050FA0EDBCFE6FFFB0EDBCFE6FF3C
:10070000FC0EDBCFE6FFFD0EDBCFE6FFFC0EDBCF02
:10071000E6FF34DE006E050EE15E0050FA0EDBCF20
:10072000E6FFFB0EDBCFE6FFFE0EDBCFE6FFFB0EA8
:10073000DBCFE6FFFC0EDBCFE6FF20DE006E050E12
:10074000E15E0050FA0EDBCFE6FFFD0EDBCFE6FFE9
:10075000FE0EDBCFE6FFFB0EDBCFE6FFFE0EDBCFB0
:10076000E6FF0CDE006E050EE15E005077DFE5521D
:10077000E7CFD9FF1200D9CFE6FFE1CFD9FF050EB1
:10078000E126030EDB6AFD0EDBCFE6FFFE0EDB503B
:10079000E552E75CE76E040EE7CFDBFFFC0EDB50B3
:1007A000E76E020EE7CFDBFF030E006EFC0EDB50A0
:1007B000E824005CDE6EDD6A030EDBCF00F0020E83
:1007C000DB50D880005401E2F3D0FB0EDBCFE6FF14
:1007D000020EDBCFE6FFFD0EDB50E552E724E66EAE
:1007E000030EDBCFE6FFFE0EDB50E552E724E66E9C
:1007F00042DDE552E552E552FB0EDBCFE6FFFD0E92
:10080000DBCFE6FF020EDB50E552E75CE66E030E3F
:10081000DBCFE6FFFE0EDB50E552E724E66E2BDD74
:10082000E552E552E552FB0EDBCFE6FF020EDBCFD1
:10083000E6FFFD0EDB50E552E724E66EFE0EDBCF51
:10084000E6FF030EDB50E552E75CE66E14DDE55291
:10085000E552E552FB0EDBCFE6FFFD0EDBCFE6FFF8
:10086000020EDB50E552E75CE66EFE0EDBCFE6FFE4
:10087000030EDB50E552E75CE66EFDDCE552E55227
:10088000E552FB0EDBCFE6FF030EDBCFE6FFFD0EEE
:10089000DB50E552E724E66E040EDBCFE6FF020EE6
:1008A000DBCFE6FFFD0EDB50E552E724E552D880B2
:1008B000E754E66EE0DCE552E552E552FB0EDBCF95
:1008C000E6FFFD0EDBCFE6FF030EDB50E552E75CF3
:1008D000E66E040EDBCFE6FF020EDBCFE6FFFD0E79
:1008E000DB50E552E724E552D880E754E66EC3DCDE
:1008F000E552E552E552FB0EDBCFE6FF030EDBCF00
:10090000E6FFFD0EDB50E552E724E66E040EDBCF7A
:10091000E6FFFD0EDBCFE6FF020EDB50E552E75CA3
:10092000E552D880E754E66EA6DCE552E552E55282
:10093000FB0EDBCFE6FFFD0EDBCFE6FF030EDB5049
:10094000E552E75CE66E040EDBCFE6FFFD0EDBCF83
:10095000E6FF020EDB50E552E75CE552D880E75433
:10096000E66E89DCE552E552E552DECF00F0DDCFE0
:1009700001F00001800E011409E0030EDB50040DAC
:10098000F350060FDE26000EDD220FD0030EDBCF64
:10099000E6FF020EDB50E552E75C040DF3500A0F50
:1009A000DE26000EDD22020EDB06030EDB2A04D754
:1009B00055DE050EE15C02E2E16AE552E16EE552C8
:1009C000E7CFD9FF1200828282908294960EE66E63
:1009D00044DCE55282808284640EE66E3EDCE552A1
:1009E000210EE66E3DD8E552900EE66E39D8E552FE
:1009F000050EE66E35D8E552130EE66E31D8E55297
:100A0000200EE66E2DD8E552960EE66E26DCE552F7
:100A10000C0EE66E25D8E552320EE66E1EDCE5526F
:100A200012008290E66AE66A72D8E552E552000149
:100A3000686B696BD890695104E6000E685D030E1F
:100A400069590DE2E66A21D8E5520A0EE66E1EECFF
:100A500001F0E5520001682B000E6923EBD712006C
:100A6000D9CFE6FFE1CFD9FF82928290190EE66ED0
:100A70001EEC01F0E552FE0EDBCFE6FF1BD8E5527F
:100A80008280E552E7CFD9FF1200D9CFE6FFE1CF50
:100A9000D9FF82828290190EE66E1EEC01F0E552BB
:100AA000FE0EDBCFE6FF06D8E5528280E552E7CFA7
:100AB000D9FF1200D9CFE6FFE1CFD9FFE652080EE9
:100AC000DF6EDFCF00F0000EE76E0018E8AE02D058
:100AD000003403D0E750D880005414E282960A0E06
:100AE000E66E1EEC01F0E552FE0EDBBE02D08298EF
:100AF00001D082888286DB50020DFE0EF3CFDBFF31
:100B0000DF06DFD7E552E552E7CFD9FF1200D9CF94
:100B1000E6FFE1CFD9FFFD0EDB50070B4009E66E83
:100B20009FDFE552FE0EDB507F0B8009E66E98DFFB
:100B3000E552E552E7CFD9FF1200D9CFE6FFE1CF6A
:100B4000D9FFE652DF6ADFCF00F0600EE76E0018D3
:100B5000E8AE02D0E73402D0E750005C10E2FE0EAF
:100B6000DBCFE6FFDFCFE6FFD2DFE552E552E66AF4
:100B7000200EE66E7ED8E552E552DF2AE4D7E55234
:100B8000E552E7CFD9FF1200D9CFE6FFE1CFD9FF79
:100B9000020EE126E66AE66ABADFE552E552DE6A4F
:100BA000DD6ADECF00F0DDCF01F0D890015004E621
:100BB000600E005C000E01581DE2E66A66DFE55239
:100BC000E66A63DFE552E66A60DFE552E66A5DDF0A
:100BD000E552E66A5ADFE552E66A57DFE552E66A11
:100BE00054DFE552E66A51DFE552DF2A010E01E3E8
:100BF000DB2AD7D7E66AE66A8ADFE552E552020EBB
:100C0000E15C02E2E16AE552E16EE552E7CFD9FF2D
:100C10001200D9CFE6FFE1CFD9FFE652DF6ADFCF7E
:100C200000F0080EE76E0018E8AE02D0E73402D0FC
:100C3000E750005C19E2DFCFE6FFFE0EDBCFE6FFF8
:100C400066DFE552E552E66A20DFE552E66A1DDF1F
:100C5000E552E66A1ADFE552E66A17DFE552E66A10
:100C600014DFE552DF2ADBD7E552E552E7CFD9FFA3
:100C70001200D9CFE6FFE1CFD9FFFE0EDBCF6AF03D
:100C8000200E00016A5D01E23BD06A517F0801E25B
:100C900037D06B6B050E6B5D30E2500E6A5D10E273
:100CA000200E6A5D050DF3CF6CF06C516B25F76A71
:100CB000700FF66E340EF7220800F5CF6DF00FD0EE
:100CC000500E6A5D050DF3CF6CF06C516B25F76A21
:100CD000600FF66E350EF7220800F5CF6DF06DC08F
:100CE000E6FFD3DEE552FD0EDB5004E06DC0E6FF0B
:100CF000CCDEE55200016B2BCDD7E66AC6DEE552AD
:100D0000E552E7CFD9FF1200D9CFE6FFE1CFD9FFF7
:100D1000E65200016F6B706B716B726BDF6AFD0ED8
:100D2000DB50DF5C07E0D8906F3770377137723770
:100D3000DF2AF5D76F836FC073F070C074F071C095
:100D400075F072C076F0746B756B766B080E1F0BC6
:100D50006FC077F070C078F071C079F072C07AF02F
:100D600008E00001D8907A33793378337733E80696
:100D7000F9E10001786B796B7A6B100E1F0B6FC075
:100D80007BF070C07CF071C07DF072C07EF008E036
:100D90000001D8907E337D337C337B33E806F9E164
:100DA00000017C6B7D6B7E6B180E1F0B6FC07FF09C
:100DB00070C080F071C081F072C082F008E0000164
:100DC000D8908233813380337F33E806F9E1000124
:100DD000806B816B826B010EE66EFE0EDBCFE6FF51
:100DE00096DEE552E5527FC0E6FF2AD8E552020EB4
:100DF000E66EFE0EDBCFE6FF8ADEE552E5527BC0F3
:100E0000E6FF1ED8E552030EE66EFE0EDBCFE6FFD0
:100E10007EDEE552E55277C0E6FF12D8E552040EB9
:100E2000E66EFE0EDBCFE6FF72DEE552E55273C0E2
:100E3000E6FF06D8E552E552E552E7CFD9FF1200AA
:100E4000D9CFE6FFE1CFD9FFE65282828290080E29
:100E5000DF6EDFCF00F0000EE76E0018E8AE02D0C4
:100E6000003403D0E750D880005415E282960A0E71
:100E7000E66E1EEC01F0E552FE0EDBB002D0829869
:100E800001D082888286DB407F0BE76EFE0EE7CFC3
:100E9000DBFFDF06DED78280E552E552E7CFD9FFE0
:100EA0001200E66A4ADEE552010EE66E46DEE552C3
:100EB000020EE66E42DEE552030EE66E3EDEE552BF
:100EC000040EE66E3ADEE552050EE66E36DEE552BB
:100ED000060EE66E32DEE552070EE66E2EDEE552B7
:100EE0001200D9CFE6FFE1CFD9FFFD0EDBCFE6FF41
:100EF000FE0EDBCFE6FF0BDEE552E552E66A200E82
:100F0000E66EB7DEE552E552E552E7CFD9FF1200B3
:100F1000E66ABBDDE552040EE66EB7DDE552020E71
:100F2000E66EB3DDE5527F0EE66EAFDDE552020EF2
:100F3000E66EABDDE552040EE66EA7DDE552E66A2D
:100F4000A4DDE552E66AA1DDE5521200100EE66E60
:100F50009CDDE552200EE66E98DDE5527F0EE66ED2
:100F600094DDE552200EE66E90DDE552100EE66E41
:100F70008CDDE552E66A89DDE552E66A86DDE552FA
:100F8000E66A83DDE5521200080EE66E7EDDE5526C
:100F90001C0EE66E7ADDE5522A0EE66E76DDE5522F
:100FA000080EE66E72DDE552080EE66E6EDDE55265
:100FB000F80EE66E6ADDE552E66A67DDE552E66A3E
:100FC00064DDE5521200080EE66E5FDDE552080EA4
:100FD000E66E5BDDE5522A0EE66E57DDE5521C0E2D
:100FE000E66E53DDE552080EE66E4FDDE552E66A29
:100FF0004CDDE552E66A49DDE552E66A46DDE5523A
:101000001200E66A42DDE552060EE66E3EDDE5526E
:10101000090EE66E3ADDE552090EE66E36DDE55262
:10102000060EE66E32DDE552E66A2FDDE552E66A2F
:101030002CDDE552E66A29DDE5521200E66A25DD7F
:10104000E552060EE66E21DDE5520F0EE66E1DDD61
:10105000E5520F0EE66E19DDE552060EE66E15DD61
:10106000E552E66A12DDE552E66A0FDDE552E66A10
:101070000CDDE5521200D9CFE6FFE1CFD9FFFD0E1E
:10108000DBCFE9FFFE0EDBCFEAFFEF5012E0FC0EF4
:10109000DBCFE6FFFD0EDBCFE9FFDB2AFE0EDBCF69
:1010A000EAFF01E3DB2AEF50E66EE3DDE552E552AD
:1010B000E6D7E552E7CFD9FF1200DACFE4FFE2CF5F
:1010C000DAFFE9CFE4FFEACFE4FFE6529EAA16D0AA
:1010D000AECFF2F0000162C0E9FF63C0EAFF622B0D
:1010E000000E6323F2C0EFFF280E625D010E63590C
:1010F00004E3000E626F010E636F9E9AF2A411D09A
:1011000080760001DB0ED46F0B0ED56FD5C02CF0AE
:101110002D6A2C50D76ED451D66ED590D592D594D9
:10112000F294E552E5CFEAFFE5CFE9FFE5CFDAFF3C
:101130001100D9CFE6FFE1CFD9FFFE0EDB50A96E3B
:10114000A69EA69CA680F40EE66E010EE66EE66AEA
:10115000E66A1FEC0FF0E552E552E552E552A85061
:1011600000D0E552E7CFD9FF1200D9CFE6FFE1CF9B
:10117000D9FFFE0EDB50A96EFD0EDB50A86EA69EB9
:10118000A684550EA76EAA0EA76EA682A1A8FED7AA
:10119000A198A694E552E7CFD9FF1200D9CFE6FF78
:1011A000E1CFD9FFFB0EDBCFE9FFFC0EDBCFEAFF7F
:1011B000EF501AE0FB0EDBCFE9FFDB2AFC0EDBCFA2
:1011C000EAFF01E3DB2AEF50E66EFD0EDBCF00F015
:1011D000DB2AFE0EDBCF01F001E3DB2A0050E66ED6
:1011E000C4DFE552E552DED7E552E7CFD9FF120062
:1011F000D9CFE6FFE1CFD9FF020EE126FD0EDBCF0E
:10120000E6FF97DFE552DE6EDD6AD9CFE9FFDACF80
:10121000EAFFEE50ED1001E11FD0DFCFE6FF4AEC10
:1012200000F0E552FD0EDB2AFE0E01E3DB2AFD0E87
:10123000DBCF00F0FE0EDBCF01F0013404E2005002
:10124000FF08000E015401E207D0D9CFE9FFDACF41
:10125000EAFFEE50ED10D2E1980EE66E3A0EE66E21
:10126000E66AE66A1FEC0FF0E552E552E552E552F8
:10127000020EE15C02E2E16AE552E16EE552E7CF7F
:10128000D9FF1200D9CFE6FFE1CFD9FF0A0EE12640
:101290000001A20EC36F010EC46FFC0EDBCF00F085
:1012A000010EE76E0018E8AE02D0003403D0E7501C
:1012B000D880005401E2EBD0FC0EDB5028E1FD0E9B
:1012C000DBCF00F0FE0EDBCF01F0060E00C0DBFF2F
:1012D000070E01C0DBFF080EDB6A090EDB6AA20EF7
:1012E000E66E010EE66ED950060FE96EDACFEAFF20
:1012F000EECFE6FFEECFE6FFEECFE6FFEFCFE6FF65
:101300007BEC19F0006E060EE15E005010D0A20ECC
:10131000E66E010EE66EFD0EDBCFE6FFFE0EDBCFC6
:10132000E6FFE1EC18F0E552E552E552E552000126
:10133000C5AD84D0A20EE66E010EE66EDEEC20F0A6
:10134000E552E552020EF3CFDBFF030EF4CFDBFFD5
:10135000DE6ADD6ADECF00F0DDCF01F0020EDBCF0A
:1013600002F0030EDBCF03F00250005C0350015883
:101370002EE2020EDBCF02F0030EDBCF03F0DE50D5
:10138000025CE96EDD500358EA6EE906000EEA5A87
:10139000A20EE926010EEA22EF50E66EFC0EDB50AB
:1013A000040F006E016A00BE0168DE50005CE96E49
:1013B000DD500158EA6EA20EE926010EEA22E5523E
:1013C000E750EF6EDF2A010E01E3DB2AC3D7DE6AA6
:1013D000DD6ADECF00F0DDCF01F0FC0EDB50050F43
:1013E000046E056A04BE0568020EDB50045C026EE2
:1013F000030EDB500558036E0250005C0350015889
:101400001DE20001C5A90BD0DECFE9FFDDCFEAFF69
:10141000A20EE926010EEA22300EEF6E0AD0DECFD0
:10142000E9FFDDCFEAFFA20EE926010EEA22200E37
:10143000EF6EDF2A010E01E3DB2ACBD7FC0EDB5077
:10144000050FE96EEA6AE9BEEA68A20EE926010E16
:10145000EA22EF6A0001C5AF0CD0FB0EDBCFE6FF3E
:10146000C3C0E6FFC4C0E6FF06DEE552E552E55222
:101470000ED0C3C0E6FFC4C0E6FFB1EC00F0E552F9
:10148000E552020EF3CFDBFF030EF4CFDBFF0A0EB3
:10149000E15C02E2E16AE552E16EE552E7CFD9FF95
:1014A0001200D9CFE6FFE1CFD9FF0E0EE126F90EEB
:1014B000DBCFDEFFDBCFDDFFF80EDBCF02F0000E6F
:1014C000E76E0218E8AE02D0023403D0E750D880AD
:1014D000025402E3070E12D0F80EDBCF03F0160E13
:1014E000E76E0318E8AE02D0033403D0E750D8808B
:1014F000035402E2170E02D0F80EDB28006E016AD8
:1015000000BE0168080E00C0DBFF090E01C0DBFF52
:10151000020EDB6A030EDB6AFB0EDBCF00F0FC0E73
:10152000DBCF01F0FD0EDBCF02F0FE0EDBCF03F0D0
:10153000246A256A266A276A00C01FF001C020F0CD
:1015400002C021F003C022F0B6EC16F0010A33E12C
:10155000F90EDBCFE9FFDB2AFA0EDBCFEAFF01E36E
:10156000DB2A2D0EEF6EFB0EDBCF00F0FC0EDBCF87
:1015700001F0FD0EDBCF02F0FE0EDBCF03F0246A9C
:10158000256A800E266EBF0E276E00C01FF001C0B8
:1015900020F002C021F003C022F0ADEC15F0FB0EEC
:1015A0001FC0DBFFFC0E20C0DBFFFD0E21C0DBFFF8
:1015B000FE0E22C0DBFFFB0EDBCF00F0FC0EDBCF0C
:1015C00001F0FD0EDBCF02F0FE0EDBCF03F0246A4C
:1015D000256A266A276A00C01FF001C020F002C0F9
:1015E00021F003C022F0ADEC16F0010A4AE1FB0E37
:1015F000DBCF00F0FC0EDBCF01F0FD0EDBCF02F005
:10160000FE0EDBCF03F0246A256A800E266E3F0EA5
:10161000276E00C01FF001C020F002C021F003C0FF
:1016200022F0B6EC16F0010A2CE1006A016A200EE5
:10163000026E410E036ED950FB0FE96EFF0EDA20E9
:10164000EA6EEECF1FF0EECF20F0EECF21F0EFCF1D
:1016500022F000C024F001C025F002C026F003C033
:1016600027F0ADEC15F022C0EDFF21C0EDFF20C04A
:10167000EDFF1FC0EFFF020EDB06030E01E2DB06EB
:10168000B6D7FB0EDBCF00F0FC0EDBCF01F0FD0E7A
:10169000DBCF02F0FE0EDBCF03F0246A256A200EBA
:1016A000266E410E276E00C01FF001C020F002C060
:1016B00021F003C022F0B6EC16F0010A2EE0FB0E7A
:1016C000DBCF00F0FC0EDBCF01F0FD0EDBCF02F034
:1016D000FE0EDBCF03F0246A256A200E266E410E33
:1016E000276E00C01FF001C020F002C021F003C02F
:1016F00022F05AEC15F0FB0E1FC0DBFFFC0E20C0E1
:10170000DBFFFD0E21C0DBFFFE0E22C0DBFF020E61
:10171000DB2A030E01E3DB2AB4D7020EDBCF00F095
:10172000030EDBCF01F0D950080FE96EDACFEAFFE4
:101730000050EE260150ED22010EF36E040EF3CFA1
:10174000DBFF050EDB6A040EDBCF20F0050EDBCFDE
:1017500021F095EC14F00A0E1FC0DBFF0B0E20C029
:10176000DBFF0C0E21C0DBFF0D0E22C0DBFF040EE1
:10177000DBCF00F0050EDBCF01F0080EDBCF02F06F
:10178000090EDBCF03F001500318E8AE02D003349A
:1017900004D00250005C035001582EE20A0EDBCF49
:1017A00000F00B0EDBCF01F00C0EDBCF02F00D0EC4
:1017B000DBCF03F0246A256A200E266E410E276EC9
:1017C00000C01FF001C020F002C021F003C022F0D1
:1017D0005AEC15F00A0E1FC0DBFF0B0E20C0DBFF1A
:1017E0000C0E21C0DBFF0D0E22C0DBFF040EDB2A36
:1017F000050E01E3DB2ABBD70A0EDBCF04F00B0E8C
:10180000DBCF05F00C0EDBCF06F00D0EDBCF07F0C3
:10181000246A256A266A400E276E04C01FF005C0A0
:1018200020F006C021F007C022F05AEC15F01FC0CE
:1018300000F020C001F021C002F022C003F0D95016
:10184000FB0FE96EFF0EDA20EA6EEECF1FF0EECF4F
:1018500020F0EECF21F0EFCF22F000C024F001C045
:1018600025F002C026F003C027F0C4EC14F022C01B
:10187000EDFF21C0EDFF20C0EDFF1FC0EFFFFB0E0D
:10188000DBCF00F0FC0EDBCF01F0FD0EDBCF02F072
:10189000FE0EDBCF03F0246A256A200E266E410E71
:1018A000276E00C01FF001C020F002C021F003C06D
:1018B00022F0B6EC16F0010A13E0FB0EDB6AFC0E18
:1018C000DB6A800EF36EFD0EF3CFDBFF3F0EF36E8F
:1018D000FE0EF3CFDBFF020EDB2A030E01E3DB2A51
:1018E000020EDBCF00F0030EDBCF01F00001800E13
:1018F00001145FE0F90EDBCFE9FFDB2AFA0EDBCF44
:10190000EAFF01E3DB2A300EEF6EF90EDBCFE9FFD1
:10191000DB2AFA0EDBCFEAFF01E3DB2A2E0EEF6EA5
:10192000080EDBCF00F0090EDBCF01F0800E0114B2
:1019300014E0020EDBCF02F0030EDBCF03F0080E43
:10194000DB50025C006E090EDB500358016E020E84
:1019500000C0DBFF030E01C0DBFF040EDB68050ED9
:10196000DB68040EDBCF00F0050EDBCF01F0020ECA
:10197000DBCF02F0030EDBCF03F003500118E8AE1B
:1019800002D0013404D00050025C0150035811E22F
:10199000F90EDBCFE9FFDB2AFA0EDBCFEAFF01E32A
:1019A000DB2A300EEF6E040EDB06050E01E2DB06CD
:1019B000D8D7040EDB6A050EDB6A040EDBCF00F01D
:1019C000050EDBCF01F0080EDBCF02F0090EDBCFF6
:1019D00003F001500318E8AE02D0033404D00250E3
:1019E000005C0350015801E3ACD0FB0EDBCF1FF0CD
:1019F000FC0EDBCF20F0FD0EDBCF21F0FE0EDBCFA7
:101A000022F047EC16F0060E20C0DBFF070E21C0C7
:101A1000DBFF300EE76E060EDBCF00F0070EDBCFEC
:101A200001F0E7500026000E0122F90EDBCFE9FF9E
:101A3000DB2AFA0EDBCFEAFF01E3DB2A00C0EFFF6F
:101A4000040EDBCF00F0050EDBCF01F0020EDB5001
:101A5000001803E1030EDB5001180BE1F90EDBCF98
:101A6000E9FFDB2AFA0EDBCFEAFF01E3DB2A2E0EC9
:101A7000EF6E060EDBCF20F0070EDBCF21F095ECEA
:101A800014F00A0E1FC0DBFF0B0E20C0DBFF0C0E94
:101A900021C0DBFF0D0E22C0DBFF1FC000F020C005
:101AA00001F021C002F022C003F0D950FB0FE96E13
:101AB000FF0EDA20EA6EEECF1FF0EECF20F0EECF71
:101AC00021F0EFCF22F000C024F001C025F002C0C9
:101AD00026F003C027F0C3EC14F022C0EDFF21C0B4
:101AE000EDFF20C0EDFF1FC0EFFF006A016A200E6E
:101AF000026E410E036ED950FB0FE96EFF0EDA2025
:101B0000EA6EEECF1FF0EECF20F0EECF21F0EFCF58
:101B100022F000C024F001C025F002C026F003C06E
:101B200027F0ADEC15F022C0EDFF21C0EDFF20C085
:101B3000EDFF1FC0EFFF040EDB2A050E01E3DB2AD9
:101B40003CD7F90EDBCFE9FFFA0EDBCFEAFFEF6AF5
:101B50000E0EE15C02E2E16AE552E16EE552E7CF8A
:101B6000D9FF1200D9CFE6FFE1CFD9FF060EE1265B
:101B70000001C59DFB0EDBCF1FF0FC0EDBCF20F07C
:101B8000FD0EDBCF21F0FE0EDBCF22F076EC16F05F
:101B90001EC0DEFF1FC0DEFF20C0DEFF21C0DDFF54
:101BA000DD52DD52FB0EDBCF04F0FC0EDBCF05F087
:101BB000FD0EDBCF06F0FE0EDBCF07F0F90EDBCF1C
:101BC00020F0FA0EDBCF21F095EC14F01FC008F0E6
:101BD00020C009F021C00AF022C00BF008C024F098
:101BE00009C025F00AC026F00BC027F004C01FF082
:101BF00005C020F006C021F007C022F0ADEC15F0C2
:101C00001FC000F020C001F021C002F022C003F08C
:101C1000F90EDBCF14F0FA0EDBCF15F0166A176A57
:101C200015AE02D01668176814C01EF015C01FF05C
:101C300016C020F017C021F0DFCF23F0010EDBCF5C
:101C400024F0020EDBCF25F0030EDBCF26F08DEC67
:101C500020F01AC010F01BC011F01CC012F01DC003
:101C600013F010C01EF011C01FF012C020F013C0FE
:101C700021F0AAEC14F01FC00CF020C00DF021C020
:101C80000EF022C00FF00CC024F00DC025F00EC0E5
:101C900026F00FC027F000C01FF001C020F002C0E6
:101CA00021F003C022F0C3EC14F047EC16F0040E50
:101CB00020C0DBFF050E21C0DBFF600EE66E010ECB
:101CC000E66ED9CFE9FFDACFEAFFEECFE6FFEECF3F
:101CD000E6FFEECFE6FFEFCFE6FF7BEC19F0006EFC
:101CE000060EE15E00500001C5AF0DD0F80EDBCF4F
:101CF000E6FF600EE66E010EE66E3BEC08F0E55284
:101D0000E552E5520CD0600EE66E010EE66EB1ECC7
:101D100000F0E552E552F3CFD2F0F4CFD3F000015A
:101D2000C5AF0AD0F80EDBCFE6FF2E0EE66E39EC1B
:101D300006F0E552E55205D02E0EE66E4AEC00F0B4
:101D4000E552F80EDBCFE6FFE66A040EDBCFE6FFD6
:101D5000050EDBCFE6FF42EC09F0E552E552E55215
:101D6000E552060EE15C02E2E16AE552E16EE552FF
:101D7000E7CFD9FF1200D9CFE6FFE1CFD9FFE65276
:101D8000800EDF6EDF50000813E2FE0EDB50DF1422
:101D900006E0310EE66E4AEC00F0E55205D0300E5A
:101DA000E66E4AEC00F0E552DF407F0BDF6EEAD7CB
:101DB000E552E552E7CFD9FF1200D9CFE6FFE1CFD8
:101DC000D9FF020EE126FE0EDB50F00BE8380F0BB8
:101DD000300FDF6EDF50390803E2070EDF24DF6EBD
:101DE000FE0EDB500F0B300FE76E010EE7CFDBFF6F
:101DF000DB5039080AE2070E006E010EDBCFE7FF69
:101E00000050E726010EE7CFDBFFDFCFE6FF4AEC0D
:101E100000F0E552010EDBCFE6FF4AEC00F0E552A0
:101E2000680EE66E4AEC00F0E552020EE15C02E25A
:101E3000E16AE552E16EE552E7CFD9FF1200D9CF52
:101E4000E6FFE1CFD9FFFB0EDBCF1FF0FC0EDBCFAF
:101E500020F0FD0EDBCF21F0FE0EDBCF22F022348E
:101E6000000E221809E6D880000E1F54000E2054E0
:101E7000000E2154000E22540CE2D950FB0FE96EE3
:101E8000FF0EDA20EA6EEE06000EEE5AEE5AEE5A19
:101E9000DAD7E552E7CFD9FF1200D9CFE6FFE1CF7D
:101EA000D9FF020EE126DE6ADD6ADECF00F0DDCF6B
:101EB00001F0FE0EDB50000101AE02D0D89003D03D
:101EC000005C000E01580AE2200EE66E4AEC00F0BB
:101ED000E552DF2A010E01E3DB2AE7D7020EE15CBF
:101EE00002E2E16AE552E16EE552E7CFD9FF120066
:101EF000D9CFE6FFE1CFD9FF020EE1268B9A100E73
:101F0000DE6EDD6ADECF00F0DDCF01F0013404E2E9
:101F100000500008000E015427E2FE0EDB50800B3B
:101F200002E1829801D08288020EE66E1EEC01F07A
:101F3000E5528286020EE66E1EEC01F0E5528296B4
:101F4000FD0EDBCF00F0FE0EDBCF01F0D8900036A7
:101F50000136FD0E00C0DBFFFE0E01C0DBFFDF0619
:101F6000010E01E2DB06CED78B8A020EE15C02E2B3
:101F7000E16AE552E16EE552E7CFD9FF1200D9CF11
:101F8000E6FFE1CFD9FFFB0EDBCFE2F0FC0EDBCFAB
:101F9000E3F0FD0EDBCFE4F0FE0EDBCFE5F0D95031
:101FA000F90FE96EFF0EDA20EA6E000ED880EE54CB
:101FB000000EED5439E20001E251016A000F006E9B
:101FC000340E012200C0E6FF01C0E6FF91DFE552BA
:101FD000E5520001E351016A000F006E250E012257
:101FE00000C0E6FF01C0E6FF83DFE552E5520001D5
:101FF000E451016A000F006E360E012200C0E6FFB8
:1020000001C0E6FF75DFE552E5520001E551016AC6
:10201000000F006E270E012200C0E6FF01C0E6FFA0
:1020200067DFE552E55238D00001E251016A000F46
:10203000006E300E012200C0E6FF01C0E6FF58DF4F
:10204000E552E5520001E351016A000F006E210ED6
:10205000012200C0E6FF01C0E6FF4ADFE552E5527B
:102060000001E451016A000F006E320E012200C02F
:10207000E6FF01C0E6FF3CDFE552E5520001E55115
:10208000016A000F006E230E012200C0E6FF01C0AE
:10209000E6FF2EDFE552E552E552E7CFD9FF120009
:1020A000600EE66E010EE66EE2C0E6FFE3C0E6FFFC
:1020B000E4C0E6FFE5C0E6FF7BEC19F0006E060E1B
:1020C000E15E0050600EE66E010EE66EB1EC00F0CF
:1020D000E552E552F3CFD2F0F4CFD3F0090EE66E1D
:1020E0004AEC00F0E552E5C0E6FF67DEE552090E76
:1020F000E66E4AEC00F0E552E4C0E6FF5EDEE55233
:10210000090EE66E4AEC00F0E552E3C0E6FF55DE4C
:10211000E552090EE66E4AEC00F0E552E2C0E6FF39
:102120004CDEE552090EE66E4AEC00F0E552E3EFB4
:1021300000F06F6A6E6A8168F90E936EC26A070ECC
:10214000C16E926E896A8268800E946E94909492A9
:10215000949494969498949A949C948E1200980EC9
:10216000E66E3A0EE66EE66AE66A69DEE552E5522A
:10217000E552E552DEDF808680880001000E626F46
:10218000010E636F62C060F063C061F00101600E18
:10219000A06F010EA16F16EC00F00C0EE66E4AEC7B
:1021A00000F0E552100EE66E270EE66EE66AE66A6D
:1021B00046DEE552E552E552E552E3EC00F0A0C1FF
:1021C000E6FFA1C1E6FFB1EC00F0E552E552F3CF26
:1021D000D2F0F4CFD3F0E3EC00F02DC100F02EC12B
:1021E00001F0026A00C0E6FF01C0E6FF02C0E6FFA0
:1021F000600EE66E010EE66EC5EC20F0036E050E75
:10220000E15E0350600EE66E010EE66EB1EC00F08A
:10221000E552E552F3CFD2F0F4CFD3F0000EE66EE4
:10222000E66AF8EC08F0E552E552E3EC00F080963F
:102230008098100EE66E270EE66EE66AE66AFFDD0F
:10224000E552E552E552E552D59CD56A100EE66E90
:10225000ECEC20F0E5520001DB0ED46F0B0ED56FD5
:10226000D5C000F0016A0050D76ED451D66ED5901B
:10227000D592D594D86BD96B640ED66FD76BE3EC3F
:1022800000F02FC100F030C101F0026A00C0E6FF8B
:1022900001C0E6FF02C0E6FF600EE66E010EE66ECC
:1022A000C5EC20F0036E050EE15E0350600EE66E95
:1022B000010EE66EB1EC00F0E552E552F3CFD2F03C
:1022C000F4CFD3F0E66AD00EE66E12DEE552E552A8
:1022D000E3EC00F031C100F032C101F0026A00C04D
:1022E000E6FF01C0E6FF02C0E6FF600EE66E010EEB
:1022F000E66EC5EC20F0036E050EE15E0350600E45
:10230000E66E010EE66EB1EC00F0E552E552F3CF59
:10231000D2F0F4CFD3F00001440EE26FDD0EE36F94
:10232000070EE46FE56B440EE66E300EE66EE0DD00
:10233000E552E552DD0EE66E210EE66ED9DDE55280
:10234000E552070EE66E320EE66ED2DDE552E5523C
:10235000E66A230EE66ECCDDE552E552E3EC00F0D2
:1023600033C100F034C101F0026A00C0E6FF01C0D1
:10237000E6FF02C0E6FF600EE66E010EE66EC5ECFB
:1023800020F0036E050EE15E0350600EE66E010E56
:10239000E66EB1EC00F0E552E552F3CFD2F0F4CFA7
:1023A000D3F000013E0EE26F360EE36F1A0EE46FBB
:1023B000E56B3E0EE66E340EE66E9ADDE552E552B2
:1023C000360EE66E250EE66E93DDE552E5521A0EE8
:1023D000E66E360EE66E8CDDE552E552E66A270EB5
:1023E000E66E86DDE552E552E66A900EE66E80DD29
:1023F000E552E552E66AC00EE66E7ADDE552E55238
:10240000E3EC00F0400EE66E420EE66E0F0EE66E56
:10241000E66A15DDE552E552E552E552E3EC00F0DF
:1024200035C100F036C101F0026A00C0E6FF01C00C
:10243000E6FF02C0E6FF600EE66E010EE66EC5EC3A
:1024400020F0036E050EE15E0350600EE66E010E95
:10245000E66EB1EC00F0E552E552F3CFD2F0F4CFE6
:10246000D3F0E66A500EE66E43DDE552E552400ECB
:10247000E66E420EE66E0F0EE66EE66AE0DCE552B0
:10248000E552E552E552E3EC00F037C100F038C107
:1024900001F0026A00C0E6FF01C0E6FF02C0E6FFED
:1024A000600EE66E010EE66EC5EC20F0036E050EC2
:1024B000E15E0350600EE66E010EE66EB1EC00F0D8
:1024C000E552E552F3CFD2F0F4CFD3F00001CE6B5A
:1024D000CF6BE26BE36BE46BE56BE66BE76BE86B92
:1024E000E96B246A500E256E430E266E470E276E4A
:1024F000E6C01FF0E7C020F0E8C021F0E9C022F0FC
:10250000C4EC14F01FC0E6F020C0E7F021C0E8F0F2
:1025100022C0E9F0E66AE66ACEC0E6FFCFC0E6FF79
:1025200042EC09F0E552E552E552E552090EE66E3D
:102530004AEC00F0E552020EE66E600EE66E010E09
:10254000E66EE6C0E6FFE7C0E6FFE8C0E6FFE9C0EA
:10255000E6FF51EC0AF0006E070EE15E0050600EDF
:10256000E66E010EE66EB1EC00F0E552E552F3CFF7
:10257000D2F0F4CFD3F0090EE66E4AEC00F0E5524B
:10258000770E006ECC0E016E2B0E026E430E036EA4
:10259000E6C024F0E7C025F0E8C026F0E9C027F047
:1025A00000C01FF001C020F002C021F003C022F0E3
:1025B000ADEC15F01FC0EEF020C0EFF021C0F0F040
:1025C00022C0F1F0020EE66E600EE66E010EE66EBF
:1025D000EEC0E6FFEFC0E6FFF0C0E6FFF1C0E6FFA9
:1025E00051EC0AF0006E070EE15E0050600EE66EE0
:1025F000010EE66EB1EC00F0E552E552F3CFD2F0F9
:10260000F4CFD3F0090EE66E4AEC00F0E552EEC0CE
:10261000E6FFEFC0E6FFF0C0E6FFF1C0E6FFB6EC74
:102620001FF0E552E552E552E5521EC000F01FC012
:1026300001F020C002F021C003F000C01FF001C073
:1026400020F002C021F003C022F076EC16F01EC08C
:10265000DAF01FC0DBF020C0DCF021C0DDF0000E9E
:10266000E66EE66ADAC0E6FFDBC0E6FFDCC0E6FF46
:10267000DDC0E6FF84DC006E060EE15E0050E66A17
:10268000900EE66E35DCE552E5520ADDF80EE66E98
:10269000240EE66E010EE66EE66A1FEC0FF0E552C0
:1026A000E552E552E5520001CE2B000ECF230A0E73
:1026B000CE5D000ECF5901E214D7CA6BCB6B62C05E
:1026C00060F063C061F0D59EF29AD08EF184F28EF4
:1026D0009D8AF28CD86BD96B6251601902E163510B
:1026E000611928E024EC00F00001C66FC651E66EC7
:1026F000E66A1FEC21F0E552E552F3CF00F0F4CF8B
:1027000001F00050011004E12E0E0001C65D12E13F
:10271000570E0001D825E96E010ED921EA6EC6C018
:10272000EFFFC6C0E6FF4AEC00F0E5520001D82BEF
:10273000000ED9230D0EC65D01E0E3D0570ED8255B
:10274000E96E010ED921EA6EEF6AE3EC00F0570E54
:10275000E66E010EE66EE9EC1BF0E552E5521EC096
:10276000EAF01FC0EBF020C0ECF021C0EDF000015A
:10277000D86BD96B020EE66E600EE66E010EE66E49
:10278000EAC0E6FFEBC0E6FFECC0E6FFEDC0E6FF07
:1027900051EC0AF0006E070EE15E0050600EE66E2E
:1027A000010EE66EB1EC00F0E552E552F3CFD2F047
:1027B000F4CFD3F0090EE66E4AEC00F0E552770E46
:1027C000006ECC0E016E2B0E026E430E036EEAC03D
:1027D00024F0EBC025F0ECC026F0EDC027F000C0DF
:1027E0001FF001C020F002C021F003C022F0ADECC8
:1027F00015F01FC0E6F020C0E7F021C0E8F022C0CD
:10280000E9F0020EE66E600EE66E010EE66EE6C0C0
:10281000E6FFE7C0E6FFE8C0E6FFE9C0E6FF51ECEF
:102820000AF0006E070EE15E0050600EE66E010ECB
:10283000E66EB1EC00F0E552E552F3CFD2F0F4CF02
:10284000D3F0090EE66E4AEC00F0E552E6C0E6FF72
:10285000E7C0E6FFE8C0E6FFE9C0E6FFB6EC1FF020
:10286000E552E552E552E5521EC000F01FC001F0EE
:1028700020C002F021C003F000C01FF001C020F012
:1028800002C021F003C022F076EC16F01EC0DAF090
:102890001FC0DBF020C0DCF021C0DDF0D880000ECE
:1028A0000001DA55000EDB55000EDC55000EDD553B
:1028B0001BE2000EE66EE66ADAC0E6FFDBC0E6FF6A
:1028C000DCC0E6FFDDC0E6FFBFEC0FF0006E060ED9
:1028D000E15E0050E66A900EE66E78EC0FF0E5528D
:1028E000E55250EC10F007D0400EE66E4AEC00F0D6
:1028F000E552E3EC00F062C060F063C061F00001FB
:10290000C66B100EE66E270EE66EE66AE66A1FECF0
:102910000FF0E552E552E552E5520001CA2B000ED8
:06292000CB23DAD6120001
:0A292600199E08D0199E21AE05D0BD
:10293000206C211EE86A2122198E21C01BF020C0C4
:102940001AF02B6A2A6A8E0E1C6E1D6A30EF17F081
:10295000199E0CD0199E21AE09D01E6C1F1E201E80
:10296000211EE86A1F2220222122198E21C01BF07D
:1029700020C01AF01FC02BF01EC02AF09E0E1C6E45
:102980001D6A30EF17F0277E196A6CEC17F084ECA3
:1029900017F019B614EF17F019A20AD019AA03D02C
:1029A00019BE14EF17F019A420EF17F01DEF17F060
:1029B00019AA05D019AC20EF17F01DEF17F019A0D8
:1029C0000AD019A808D019BE04D019A402D029EF42
:1029D00017F02DEF17F02A6A1D6A2750225C296E26
:1029E00010E31FC02BF020C01AF021C01BF022C042
:1029F00028F024C01FF025C020F026C021F0193A8D
:102A000009D024C02BF025C01AF026C01BF027C027
:102A100028F0296C199E19BC198E28C01CF019B019
:102A20005CEF17F01A0E29605CEF17F01C6A226A3F
:102A300019A408D01F6C201E211E221EE86A202225
:102A40002122222219AC08D02B6C1A1E1B1E1C1E20
:102A5000E86A1A221B221C221E6A295207E022342D
:102A6000213220321F321E32292EF9D71F502B2639
:102A700020501A2221501B2222501C221EC02AF054
:102A8000199E1CAE0BD02A6C2B1E1A1E1B1E1C1E60
:102A9000E86A2B221A221B221C22198E1CA006D0A7
:102AA000D8801B321A322B322A32282A28C01CF036
:102AB00030EF17F0196A6CEC17F084EC17F019B6C8
:102AC00014EF17F019A205D019BA14EF17F01BEF85
:102AD00017F019BA27EF17F019A005D019B814EF9D
:102AE00017F027EF17F019B81BEF17F01D6A7F0ECC
:102AF00022241C6EE86A1D2227501C5EE86A1D5ABB
:102B00001A0E286E226A2A6A2B6A1A6A1B6A2450D5
:102B10001F5E2550205A2650215A000E225A09E7DE
:102B200024501F262550202226502122000E22222A
:102B300001D02A8AD8901F36203621362236D890E6
:102B40002A362B361A361B36282EE1D72150201074
:102B50001F10D8A42A8A30EF17F0196A6CEC17F00E
:102B600084EC17F019B614EF17F019A205D019B8B4
:102B700014EF17F01BEF17F019AA05D019B014EFD6
:102B800017F01BEF17F019B002D019A802D027EFE9
:102B900017F01D6A275022241C6EE86A1D227E0E43
:102BA0001C5EE86A1D5A2A6A2B6A1A6A1B6A26503A
:102BB0002102F4CF1BF0F3CF1AF025502102F3507D
:102BC0002B26F4501A22000E1B2226502002F3500E
:102BD0002B26F4501A22000E1B2224502102F350FF
:102BE0002A26F4502B22000E1A221B2225502002E6
:102BF000F3502A26F4502B22000E1A221B222650B4
:102C00001F02F3502A26F4502B22000E1A221B22F8
:102C100024502002F4502A26000E2B221A221B22B6
:102C200025501F02F4502A26000E2B221A221B22A6
:102C300030EF17F021C02BF020C02AF020502502E1
:102C4000F4CF1FF0F3CF1EF021502602F4CF21F075
:102C5000F3CF20F02502F3501F26F4502022E86A1B
:102C600021222A502602F3501F26F4502022E86A1F
:102C7000212226AE40EF16F02A50205E2B50215A1A
:102C80002BAE000C2550205E2650215A000C196AEC
:102C90006CEC17F019B651EF16F019A20ED019B45A
:102CA00005D07F0E216EFF0E206E1FD0800E216E8C
:102CB000206A1BD0216A206A18D019B0FBD78F0E6A
:102CC0002260EDD77E0E2264F5D78E0E225C05E0E1
:102CD000D89021322032222AF8D719A406D0206CAD
:102CE000211EE86A212221AEE5D71200196A6CEC98
:102CF00017F019B680EF16F019A20FD019B407D04B
:102D00007F0E216EFF0E206E1F6E1E6E25D0800E70
:102D1000216E01D0216A000EF6D719B0FBD71E6ACA
:102D20009F0E2260EBD77E0E2264F4D79E0E225CAB
:102D300007E0D890213220321F321E32222AF6D7E5
:102D400019A40AD01E6C1F1E201E211EE86A1F2215
:102D50002022212221AEDED71200BFEC16F019B6D8
:102D6000000C19B0000C19B4000C010CBFEC16F0EB
:102D700019B6000C19B0000C19A4000C010C196A4A
:102D80006CEC17F084EC17F019B6120019AE08D0ED
:102D900019A004D019A802D01980120019901200AD
:102DA0002750225C0BE12650215C08E12550205C75
:102DB00005E124501F5C02E119801200D8A002D066
:102DC000198E10D0225027C022F0276E215026C025
:102DD00021F0266E205025C020F0256E1F5024C003
:102DE0001FF0246E2750225C10E0FF0F09E01990BD
:102DF00019B403D019AE1984120019AE1994120037
:102E0000272AD89026322532243224501F5E25509E
:102E1000205A2650215A21BEEAD7D8901F36203694
:102E20002136222EF8D7C8D77F0E226EFF0E216ED4
:102E3000206E1F6E12007F0E19BEFF0E226E02D092
:102E40007F0E226E800E216E206A1F6AF3D719AEA4
:102E500004D0800E226E216AF7D7226A216AF4D745
:102E60001B501A102B102A10F8E01DBEF0D71BBE05
:102E70000CD01C501D10EBE0D8902A362B361A3699
:102E80001B361C06D8A01D06F2D71D50D4E11C2805
:102E9000D2E02AAE11D07F0E2A1402E12BA00CD072
:102EA0002B2AE86A1A221B2207E3D8801B321A3227
:102EB0002B321C2A1C28BFE01C50C9E02BC01FF07D
:102EC0001AC020F01B34216E1C30226E2132229E4B
:102ED00019BE228E1AEF17F02136223602E319842A
:102EE000197E06E11980226A216A206A1F6A12008F
:102EF000222803E0D88021321200D890213202E14A
:102F000019821200198612002636273602E3198C20
:102F1000197E06E11988276A266A256A246A120042
:102F2000272803E0D88026321200D8902632EAE122
:042F3000198A1200E8
:0C2F3400FF0EE3CFEAFFE552FF0EE3CFF3
:102F4000E9FFE552E66AE66AD9CFE6FFDACFE6FFA7
:102F5000FC0EE124D96EFF0EE220DA6EE66AE66A24
:102F6000E66A200EEF5C06E0090EEF5C03E0EF6618
:102F700003D03FD0EE50F5D72D0EEF5C03E1FF0EEE
:102F8000E32A03D02B0EEF5C01E1EE502F0EEF642D
:102F900024D03A0EEF6021D0D890F90EE336FA0E25
:102FA000E336FD0EDECFE3FFFE0EDDCFE3FFD8906C
:102FB000F90EE336FA0EE336D890F90EE336FA0E40
:102FC000E336FD0EE350DE26FE0EE350DD22300E2A
:102FD000EE5CDE26000EDD22D9D7FF0EE3CFE8FF40
:102FE000E85207E0F90EE31EE32AFA0ED8B4E3062E
:102FF000E31EE552E552E552FF0EE3CFDAFFE5525C
:10300000FF0EE3CFD9FFE552E1CFE9FFE2CFEAFFC0
:10301000ED52ED52EECFF3FFEFCFF4FF1200D9CF18
:10302000E6FFDACFE6FFE66AE66AE66AE66AE66A9D
:10303000E66AE66AE66AE66AE66AF20EE3CFE9FF66
:10304000F30EE3CFEAFF200EEF5C06E0090EEF5C23
:1030500003E0EF6603D07BD0EE50F5D72D0EEF5C8A
:1030600003E1FF0EE38003D02B0EEF5C01E1EE5095
:10307000FA0EE124D96EFF0EE220DA6E2E0EEF5C1E
:1030800004E1FF0EE382EE52F9D72F0EEF6449D030
:103090003A0EEF6046D0D890FA0EE336FB0EE336D8
:1030A000FC0EE336FD0EE336F60EDECFE3FFF70E41
:1030B000DECFE3FFF80EDECFE3FFF90EDDCFE3FF57
:1030C000DD52DD52D890FA0EE336FB0EE336FC0EED
:1030D000E336FD0EE336D890FA0EE336FB0EE33608
:1030E000FC0EE336FD0EE336F60EE350DE26F70E59
:1030F000E350DE22F80EE350DE22F90EE350DD222B
:10310000DD52DD52300EEE5CDE26000EDE22DE22C7
:10311000DD22DD52DD52FF0EE3A2B0D7FE0EE30644
:10312000ADD7FF0EE3A013D0FA0EE31EFB0EE31E95
:10313000FC0EE31EFD0EE31EFA0EE32A08E1FB0E71
:10314000E32A05E1FC0EE32A02E1FD0EE32AF20E7A
:10315000E9CFE3FFF30EEACFE3FFEE0EE3CFD9FFB3
:10316000EF0EE3CFDAFFFA0EE3CFDEFFFB0EE3CF85
:10317000DEFFFC0EE3CFDEFFFD0EE3CFDDFFDD5211
:10318000DD52F00EE3CFD9FFF10EE3CFDAFFFE0EF2
:10319000E3CFDFFFF20EE124E96EFF0EE220EA6EDC
:1031A000F60EE126FF0EE222FF0EE3CFDAFFE55234
:1031B000FF0EE3CFD9FFE552EECFF3FFEFCFF4FFE1
:1031C0001200D9CFE6FFDACFE6FFFA0EE3CFD9FF40
:1031D000FB0EE3CFDAFFFD0EE35209E72D0EDE6EA4
:1031E000FC0EE31EE32AFD0ED8B4E306E31EE6520E
:1031F000E652E652FD0EE124E76EFF0EE220E46E99
:10320000E652F70EE3CFE6FFF70EE3CFE6FF51EC11
:1032100019F0F90EE124E96EFF0EE220EA6E41ECAE
:1032200019F00AE13EEC19F009E141EC19F008E16E
:103230003EEC19F007E108D04CEC19F047EC19F01E
:103240004CEC19F047EC19F04CEC19F0DE6AF90E71
:10325000E126FF0EE222FF0EE3CFDAFFE552FF0E7A
:10326000E3CFD9FFE552FC0EE124E96EFF0EE22028
:10327000EA6EEECFF3FFEFCFF4FF1200EF380F0B43
:103280001200EF500F0B02E1EE52D8841200EF381B
:103290000F0B300FDE6E1200EE500F0B300FDE6E94
:1032A0001200FC0EE3CFE9FFFD0EE3CFEAFF100EA4
:1032B000E66EEE6AEE6AEF6AD890FD0EE336FE0E19
:1032C000E336ED36ED36EF36FF0EE30609E072EC3D
:1032D00019F0EE5272EC19F0EE5272EC19F0EDD7D3
:1032E000E56E1200030EEF24E8B6EF6E300EEF2409
:1032F000E8BEEF6E000CD9CFE6FFDACFE6FFF80E9E
:10330000E3CFD9FFF90EE3CFDAFFE652E652E652F9
:10331000E652E652FB0EE124E76EFF0EE220E46E79
:10332000E652F30EE3CFE6FFF30EE3CFE6FFF30E34
:10333000E3CFE6FFF30EE3CFE6FF00EC1AF0F50E65
:10334000E124E96EFF0EE220EA6EEDEC19F019E1DE
:10335000F0EC19F018E1EDEC19F017E1F0EC19F0D0
:1033600016E1EDEC19F015E1F0EC19F014E1EDECDB
:1033700019F013E1F0EC19F012E1EDEC19F011E1A4
:1033800012D0F6EC19F0FBEC19F0F6EC19F0FBECAE
:1033900019F0F6EC19F0FBEC19F0F6EC19F0FBEC77
:1033A00019F0F6EC19F0FBEC19F0DE6AF50EE126E7
:1033B000FF0EE222FF0EE3CFDAFFE552FF0EE3CF6E
:1033C000D9FFE552FA0EE124E96EFF0EE220EA6E23
:1033D000EECFF3FFEFCFF4FF1200EF380F0B120028
:1033E000EF500F0B02E1EE52D8841200EF380F0BB2
:1033F000300FDE6E1200EE500F0B300FDE6E12003B
:10340000FA0EE3CFE9FFFB0EE3CFEAFF200EE66EF4
:10341000EE6AEE6AEE6AEE6AEF6AD890FB0EE33669
:10342000FC0EE336FD0EE336FE0EE336ED36ED36EA
:10343000ED36ED36EF36FF0EE3060FE02FEC1AF017
:10344000EE522FEC1AF0EE522FEC1AF0EE522FEC57
:103450001AF0EE522FEC1AF0E1D7E56E1200030ECF
:10346000EF24E8B6EF6E300EEF24E8BEEF6E000CEE
:10347000000000000000005F0000000700070014CB
:103480007F147F14242A7F2A12231308646236498A
:103490005522500005030000001C2241000041227B
:1034A0001C0014083E081408083E080800503000AC
:1034B00000080808080800606000002010080402E6
:1034C0003E5149453E00427F4000426151494621FC
:1034D00041454B311814127F1027454545393C4A68
:1034E00049493001710905033649494936064949B8
:1034F000291E00363600000056360000081422410E
:103500000014141414140041221408020151090675
:10351000324979413E7E1111117E7F494949363E3B
:10352000414141227F4141221C7F494949417F0954
:103530000909013E4149497A7F0808087F00417F17
:1035400041002040413F017F081422417F4040401C
:10355000407F020C027F7F0408107F3E4141413EC4
:103560007F090909063E4151215E7F091929464616
:103570004949493101017F01013F4040403F1F203F
:1035800040201F3F4038403F631408146307087011
:1035900008076151494543007F414100020408107A
:1035A000200041417F0004020102044040404040AD
:1035B000000102040020545454787F4844443838B1
:1035C00044444420384444487F3854545418087EB6
:1035D0000901020C5252523E7F0804047800447DD7
:1035E00040002040443D007F1028440000417F40BF
:1035F000007C041804787C08040478384444443877
:103600007C14141408081414187C7C08040408485A
:1036100054545420043F4440203C4040207C1C2013
:1036200040201C3C4030403C44281028440C505062
:10363000503C4464544C44000836410000007F0074
:103640000000413608001008081008784641467806
:103650004331383A203138463235325F4444535F83
:103660004144393833355F52533233325F31313070
:103670003932392E630D00496E697420414439385E
:1036800033350D004672657130203D2033303048AF
:103690007A0D004672657131203D2031304B687AD9
:1036A0000D0053656C6563742046726571300D00C2
:1036B00053657175656E636520656E2031302073CA
:1036C000746570732064652035304B7A0D0063613A
:1036D000722072656375203A00496E697420312E3C
:1036E0002E2E2E2E2E2E2E2E2E2E2E0D00496E69B3
:1036F0007420322E2E2E2E2E2E2E2E2E2E2E2E0DCF
:1037000000536F72746965204E6F726D616C652035
:103710006465205072670045534320706F757220B6
:10372000736F727469720D00313846323538204E2D
:103730006F6B6961204C4344002044445320414452
:10374000393833352020202020003239207365702D
:103750007420323031312020202000313233343592
:103760003637383930313233343536004D504C41EC
:1037700042204331382E2E2E2E2E2E2E0020206E4B
:103780006F6B696120333431302E2E2E2E002E2E99
:103790002E2E2E2E2E2E2E2E2E2E2E2E2E2E00376E
:1037A00020204C415354204C494E45202E2E2E00B3
:1037B0002020202020202020202020202020202009
:1037C000002E2E2E2E2E2E2E2E2E2E2E2E2E2E2E47
:0237D0002E00C9
:0E37D200D9CFE6FFDACFE6FFE1CFD9FFE2CF95
:1037E000DAFF100EE12402E3E168E652E16E0F0E0B
:1037F000DB6AD950020FE66E000EDA20E66ED95071
:10380000060FE66E000EDA20E66EFC0EDBCFE6FF5A
:10381000FD0EDBCFE6FF0FEC18F0006E060EE15C4C
:1038200002E2E16AE552E16E0050F3CFDEFFF4CF31
:10383000DDFFDECFE9FFDDCFEAFFEF50DF0B45080C
:1038400014E1DF2A010E01E3DB2ADECFE6FFDDCF44
:10385000E6FF9AEC17F0E552E552060EDBCFE7FFE4
:10386000F350E726060EE7CFDBFF020EDBCF00F0BA
:10387000030EDBCF01F0040EDBCF02F0050E03D9FF
:10388000AAEC14F0F3D8060EDB5001E190D006D973
:1038900000340BE3010EF36E0F0EF3CFDBFF060EC9
:1038A000DB50FF0D060EF3CFDBFF0B0EDB6A0C0EB9
:1038B000DB6A800EF36E0D0EF3CFDBFF3F0EF36E6F
:1038C0000E0EF3CFDBFFEAD8140EE76E0018E8AE59
:1038D00002D0E73402D0E750005C0BE397D8EC0E3F
:1038E000246E780E256EAD0E266E600E77D8140EFF
:1038F000B3D8D4D80A0EE76E0018E8AE02D0E73489
:1039000002D0E750005C0BE381D8F90E246E020E62
:10391000256E150E266E500E61D80A0E9DD8BED8A3
:10392000050EE76E0018E8AE02D0E73402D0E7508B
:10393000005C0AE36BD8246A500E256EC30E266E17
:10394000470E4CD8050E88D8A9D8020EE76E00188D
:10395000E8AE02D0E73402D0E750005C09E356D865
:10396000246A256AC80E266E420E38D8020EEBD79E
:1039700095D8010EE76E0018E8AE02D0E73402D009
:10398000E750005C09E342D8246A256A200E266EBF
:10399000410E24D8060EDB060F0EDB5004E043D8A0
:1039A0005AEC15F003D03FD8ADEC15F05FD8070EF8
:1039B000DBCF00F0080EDBCF01F0090EDBCF02F009
:1039C0000A0E61D8100EE15C02E2E16AE552E16E96
:1039D000E552E5CFDAFFE7CFD9FF1200276E00C02E
:1039E0001FF001C020F002C021F003C022F0ADECB6
:1039F00015F00B0E1FC0DBFF0C0E20C0DBFF0D0E01
:103A000021C0DBFF0E0E22C0DBFF12000B0EDBCF4E
:103A100000F00C0EDBCF01F00D0EDBCF02F00E0E2E
:103A2000DBCF03F01200070EDBCF1FF0080EDBCF59
:103A300020F0090EDBCF21F00A0EDBCF22F00B0EB7
:103A4000DBCF24F00C0EDBCF25F00D0EDBCF26F004
:103A50000E0EDBCF27F01200006E060EDBCFE7FF65
:103A60000050E75E060EE7CFDBFF1200070E1FC017
:103A7000DBFF080E20C0DBFF090E21C0DBFF0A0EB2
:103A800022C0DBFF1200DBCF03F000C01EF001C03C
:103A90001FF002C020F003C021F01200060EDBCFA1
:043AA00000F0120020
:0C3AA400D9CFE6FFDACFE6FFE1CFD9FF73
:103AB000E2CFDAFF130EE12402E3E168E652E16EA1
:103AC0000C0EDB6AD950FA0FE96EFF0EDA20EA6EAF
:103AD000080EEECFDBFF090EEECFDBFF0A0EEECFB6
:103AE000DBFF0B0EEECFDBFF1FD9D950080F17D924
:103AF000EECFE6FFEECFE6FFEECFE6FFEFCFE6FF3D
:103B00009BEC1EF0006E060EE15C02E2E16AE552FB
:103B1000E16E0050DF6E020EDF5C01E0BCD0050EEE
:103B2000DBCF02F0060EDBCF03F0F80EDB50025CB9
:103B3000006EF90EDB500358016E7F0E005E000E22
:103B4000015A0D0E00C0DBFF0E0E01C0DBFF0D0E93
:103B50000E0EDBCF01F00001800E01140AE0010E11
:103B6000F36E0C0EF3CFDBFF070EDB5001E098D0B5
:103B70009DD00D0EDBCF00F00E0EDBCF01F0D89004
:103B8000015004E6170E005C000E015801E39ED0C0
:103B9000046805687F0E066E076A0D0EDB501F0B6A
:103BA00004C000F005C001F006C002F007C003F039
:103BB00007E0D8900332023201320032E806F9E120
:103BC0000F0E00C0DBFF100E01C0DBFF110E02C0A4
:103BD000DBFF120E03C0DBFF0F0EDBCF00F0100E79
:103BE000DBCF01F0110EDBCF02F0120EDBCF03F0C2
:103BF000D950010F94D8EE500016EE500116EE5039
:103C00000216EE500316005001100210031002E1DC
:103C1000000E01D0010EE76E0C0EE7CFDBFFDB508C
:103C200055E0046A056A800E066E076A010E086E8A
:103C3000096A0A6A0B6AD9500F0F71D8EE5008262C
:103C4000EE500922EE500A22EE500B220850045C7E
:103C5000006E09500558016E0A500658026E0B504E
:103C60000758036ED950010F5AD80050EE16015074
:103C7000EE160250EE160350EE16D950080FE66EFF
:103C8000000EDA20E66E50D829EC1FF0E552E5521E
:103C9000E552E5521BD0DF0419E1070EDB5006E0C8
:103CA000006A016A026A800E036E04D0006A016A2B
:103CB000026A036A080E00C0DBFF090E01C0DBFFC9
:103CC0000A0E02C0DBFF0B0E03C0DBFFF60EDBCFDC
:103CD000E9FFF70EDBCFEAFF0C0EDBCFEFFF080E9C
:103CE000DBCF00F0090EDBCF01F00A0EDBCF02F0D4
:103CF0000B0EDBCF03F000C01EF001C01FF002C0AE
:103D000020F003C021F0130EE15C02E2E16AE5520B
:103D1000E16EE552E5CFDAFFE7CFD9FF1200E96E99
:103D2000000EDA20EA6E1200D950010FE66E000E86
:063D3000DA20E66E12002D
:0A3D3600D9CFE6FFDACFE6FFE1CFB8
:103D4000D9FFE2CFDAFFE652006801687F0E026E0B
:103D5000036AD950FA0FE96EFF0EDA20EA6EEE50D0
:103D60000016EE500116EE500216EE5003166AD8F9
:103D700000C0EEFF01C0EEFF02C0EEFF03C0EEFF89
:103D8000FD0EDB50800B02E0010E01D0000EE66E4E
:103D900059D8060EE926000EEA22E552E750EF6EEA
:103DA000FC0EDBCF00F0FD0EDBCF01F0D89000362B
:103DB0000136FC0E00C0DBFFFD0E01C0DBFFDB5057
:103DC000E66E40D8040EE926000EEA22E552E750DE
:103DD000EE6EED6AFD0EDB50006E016AFF0E0018FC
:103DE00018E1015016E12ED8EECF00F0EECF01F031
:103DF000EECF02F0EFCF03F00050011002100310DD
:103E000006E0210E0001F76FF86B800E0BD0040E58
:103E100009D0FD0EDB5008E115D8EE6AEE6AEE6AB5
:103E2000EE6A010EDF6E06D0020EDF6E0BD8EE5288
:103E3000EE52EE8EDF50E552E552E5CFDAFFE7CFE6
:103E4000D9FF1200F80EDBCFE9FFF90EDBCFEAFF56
:023E500012005E
:0E3E5200D9CFE6FFDACFE6FFE1CFD9FFE2CF0E
:103E6000DAFF5BD8013411E20050FE08000E015465
:103E70000CE276D805E06CD8800EEE6EEE6847D086
:103E800067D8800EEE6E7F0E0ED047D8D8900150C6
:103E900004E6010E005C000E01580BE261D805E05B
:103EA00057D8EE6A800EEE6E32D052D8EE6AEE6AC5
:103EB0002ED047D8EECF00F0EECF01F0EECF02F0DB
:103EC000EFCF03F032D800C0EEFF01C0EEFF02C01A
:103ED000EEFF03C0EEFF21D80050010B05E025D80E
:103EE000020E3AD8EF8E04D020D8020E35D8EF9EBD
:103EF00014D8D8900132003218D8030E2DD800C043
:103F0000EFFF1AD804E011D8030E26D8EF8EE55241
:103F1000E5CFDAFFE7CFD9FF120013D8040E1CD883
:103F2000EECF00F0EFCF01F01200FA0EDBCFE9FF89
:103F3000FB0EDBCFEAFF120004D8060E0DD8EF50BF
:103F40001200FC0EDBCFE9FFFD0EDBCFEAFF120013
:103F5000ECDFEE6AEE6A1200E926000EEA22120099
:0C3F6000220E0001F76FF86B9CEF1FF0C1
:043F6C00D9CFE6FFC4
:103F7000DACFE6FFE1CFD9FFE2CFDAFF060EE12488
:103F800002E3E168E652E16ED950050FE66E000EDD
:103F9000DA20E66E000EE66EE66AD950FA0FE96E98
:103FA000FF0EDA20EA6EEECFE6FFEECFE6FFEECFB1
:103FB000E6FFEFCFE6FF52EC1DF0006E080EE15C6D
:103FC00002E2E16AE552E16E0050010E1EC0DBFF25
:103FD000020E1FC0DBFF030E20C0DBFF040E21C05A
:103FE000DBFF050EDB502AE0040EDB50800B26E1E0
:103FF000006A016A800E026E3F0E036ED950010FF7
:10400000E96E000EDA20EA6EEECF1FF0EECF20F060
:10401000EECF21F0EFCF22F000C024F001C025F058
:1040200002C026F003C027F0C4EC14F022C0EDFF5C
:1040300021C0EDFF20C0EDFF1FC0EFFF010EDBCF61
:1040400000F0020EDBCF01F0030EDBCF02F0040E16
:10405000DBCF03F000C01EF001C01FF002C020F053
:1040600003C021F0060EE15C02E2E16AE552E16E76
:0C407000E552E5CFDAFFE7CFD9FF1200E0
:04407C001E0EF66EB0
:10408000000EF76E000EF86E01010900F550BC6FCE
:104090000900F550BD6F03E1BC6701D03DD00900B8
:1040A000F550B76F0900F550B86F0900F550B96FBA
:1040B00009000900F550E96E0900F550EA6E0900A3
:1040C00009000900F550BA6F0900F550BB6F0900EF
:1040D0000900F6CFBEF1F7CFBFF1F8CFC0F1B7C1FD
:1040E000F6FFB8C1F7FFB9C1F8FF0101BA5302E109
:1040F000BB5307E00900F550EE6EBA07F8E2BB07C4
:10410000F9D7BEC1F6FFBFC1F7FFC0C1F8FF01017B
:0A411000BC07000EBD5BBFD7120014
:06411A001E502302F3CF4A
:104120001AF0F4CF1BF02402F3501B26000EF420EB
:104130001C6E1E502502F3501C26000EF4201D6E2E
:104140001E502602F3501D261F502302F3501B263B
:10415000F4501C22000E1D221F502402F3501C2676
:10416000F4501D221F502502F3501D26205023021B
:10417000F3501C26F4501D2220502402F3501D261B
:0A41800021502302F3501D26120007
:06418A00FB0EE3CFF6FF7F
:10419000FC0EE3CFF7FFFD0EE3CFF8FFFE0EE3CFFB
:1041A000E9FFFF0EE3CFEAFFE9CFF3FFEACFF4FF29
:1041B0000900F5CFEFFFEE66FBD71200FE0EE3CF4E
:1041C000E9FFFF0EE3CFEAFFF36AF46AEE5203E081
:0841D000F34AF42AFBD71200A8
:0841D800D9CFE6FFDACFE6FFC4
:1041E000E1CFD9FFE2CFDAFFFD0EDB507F0BD56EBA
:1041F000D76AD66AF294FD0EDBAE02D0F28A01D005
:10420000F29AD58EE552E5CFDAFFE7CFD9FF12005B
:10421000FF0EE3502F6EEF0E01D0F30EE76EE72E88
:104220000FEF21F00C0E2E6EE76AE72E15EF21F04E
:0E4230002E2E14EF21F02F2E0DEF21F0120094
:02423E00F36A21
:10424000F46AFF0EE124E96EFF0EE220EA6EED66ED
:1042500007D02F0EEF6404D03A0EEF6001D0F32A9E
:0242600012004A
:0E426200000EF36E00EE00F0060E01D8120002
:10427000EA6002D0EE6AFCD7F350E9601200EE6A01
:02428000FCD769
:0E42820015EE00F025EE00F0F86A199C3EECF7
:0E42900020F003EC00F0AFEC10F0FBD71200B2
:02429E003132BB
:1042A000333435363738393031323334353600002F
:1042B00000000000000000000000000000000000FE
:1042C0000000000000000000000000503677368437
:1042D000369336A236B036CE36D936ED360137179C
:1042E00037283739374A375B376C377D378E379FFA
:1042F00037B037C137303030303030303000505286
:104300004F4A45543A204144393833355F313846B5
:104310002E6D6370200D0000000000000000000002
:10432000000000000000000000000000000000008D
:10433000000000000000000000000000000060011C
:104340003132333435363738393031323334350061
:05435000000000000068
:020000040030CA
:01000100FA04
:01000200F409
:01000300FEFE
:01000600FBFE
:0200000400F00A
:10000000506F727420436F6D20313932303062206E
:100010002620496E697420484152442E2E2E2E000F
:100020002E2E2E2E2E2E2E2E2E2E2E2E2E2E2E2EF0
:1000300020203C4553433E206578697420202000F1
:100040002E2E2E2E2E2E2E2E2E2E2E2E2E2E2E2ED0
:100050002E2E2E2E2E2E2E2E2E2E2E2E2E2E2000FC
:100060002E2E2E2E2E2E2E2E2E2E2E2E2E2E2E2EB0
:100070002E2E2E2E2E2E2E2E2E2E2E2E2E2E0D00EF
:10008000313846323532206176656320626F6F7495
:100090006C6F6164657220202020202020200D00DC
:1000A0007061756C666A756A6F40667265652E660A
:1000B00072202020202020202020202020200D0021
:1000C0004D504C4142204944452056382E36332E5F
:1000D0002E2E2E2E2E2E2E2E2E2E2E2E2E200D009D
:1000E0004D504C4142204331382076332E33372E49
:1000F0003031202E2E2E2E2E2E2E2E2E0D0A0000CA
:00000001FF
